:020000040000FA
:100000000029C83093007C309400000000000000FC
:1000100000000000940B052800000000930B03284B
:10002000003405309500950B1328000008000730B8
:100030009500950B1928000008000D08890083160B
:10004000081483120808900083160030860083127B
:10005000100886008514172085108316FF3086004F
:100060008312080016089A009A0E19081A078F00C2
:1000700083160030860083120F08860005141720AF
:1000800005108316FF308600831208001608013E13
:1000900098000301980B4D284F28043E4A28170763
:1000A0008D0008000830910085110000000000005C
:1000B00000000000000011200E185F28622885153E
:1000C000112065288511112065288E0C910B5C2864
:0800D000851511201120080024
:1002000008308500003086008316103085000030ED
:10021000860083120A30920000308F008F0E01207A
:1002200001200F0886000514172005108F0E8F0A75
:10023000920B0E298316FF3086008312C0308C008B
:1002400000309600013097000130990046201D20B3
:100250003220061C2F291720061C2F295329861C03
:1002600035291720861C35298129061D3B29172091
:10027000061D3B299529861D41291720861D4129E8
:10028000A929061E47291720061E4729BD29861EB3
:100290004D291720861E4D296A29051E2929172058
:1002A000051E2929D12916080311003C03196329C9
:1002B0000130960246200C088E0052200D088E0058
:1002C00052201D203220172006186329012006180D
:1002D0006329292916080311093C03197A290130D9
:1002E000960746200C088E0052200D088E005220E2
:1002F0001D2032201720861A7A290120861A7A2991
:1003000029290130970046200C088E0052200D0844
:100310008E0052201D2001309900322017208618AF
:100320008E29012086188E2929290230970046201F
:100330000C088E0052200D088E0052201D20023025
:100340009900322017200619A22901200619A22996
:1003500029290330970046200C088E0052200D08F2
:100360008E0052201D20043099003220172086195B
:10037000B62901208619B62929290430970046207C
:100380000C088E0052200D088E0052201D200830CF
:10039000990032201720061ACA290120061ACA29F4
:1003A000292905151720051AD2291720051AD2293F
:1003B000061CDE291720061CDE290E2A861CE429CD
:1003C0001720861CE4291B2A061DEA291720061D72
:1003D000EA29282A861DF0291720861DF029352AAA
:1003E000061EF6291720061EF629422A861EFC291B
:1003F0001720861EFC294F2A061F022A1720061FD7
:10040000022A5C2A861F082A1720861F082A692AC2
:10041000051ED8291720051ED829762A1018122A59
:100420001014132A1010242017200618142A012053
:100430000618142AD82990181F2A9014202A9010E0
:10044000242017208618212A01208618212AD8293D
:1004500010192C2A10152D2A1011242017200619E6
:100460002E2A012006192E2AD8299019392A9015EA
:100470003A2A90112420172086193B2A0120861938
:100480003B2AD829101A462A1016472A101224206F
:100490001720061A482A0120061A482AD829901A35
:1004A000532A9016542A901224201720861A552A6F
:1004B0000120861A552AD829101B602A1017612A94
:1004C000101324201720061B622A0120061B622A13
:1004D000D829901B6D2A90176E2A9013242017207C
:1004E000861B6F2A0120861B6F2AD829000017203F
:1004F000051A772A0120051A772A0D0889001008A5
:1005000088008316081555308900AA3089008814A0
:0E05100017208818892A08118312051129293D
:02400E00F13F80
:00000001FF
